:100000000C9410030C9457030C9457030C9457034F
:100010000C9457030C9457030C9457030C945703F8
:100020000C9457030C9457030C94750C0C94470DC7
:100030000C9457030C9457030C9457030C945703D8
:100040000C9457030C94BB210C9457030C94570346
:100050000C9457030C944D1B0C9457030C945703AA
:100060000C9457030C9457030C9457030C945703A8
:100070000C9457030C9457030C9457030C94570398
:100080000C9457030C9457030C9457030C94570388
:100090000C9457030C9457030C9457030C94570378
:1000A0000C9457030C9457030C945703B40DD60DBE
:1000B000C90ED60DC90E1B0E3E0EC90E930EA60E0E
:1000C00090119011BF11BF1102123C124914491432
:1000D000551249144A134A131D144914491434146F
:1000E00000F001F002F0F0A3F0A42B00340039007E
:1000F000E100E00000001E00140004001D00E2000A
:10010000007F1F001A0016001B0003522800200069
:10011000080007000600E3002C002100150009007C
:10012000190064002D00220017000A0005000000DD
:1001300050002E004A0000000154000052002E0022
:100140004D00000002540000510023001C000B0071
:10015000110000004F00240018000D001000E60000
:100160002D0025000C000E003600E7002C002600B4
:1001700012000F003700035228002700130033003D
:100180003800E60000772A002F003100E500E40087
:1001900000002B0006003900E100E00000001E0016
:1001A000130007003400E200007F1F0017000B005F
:1001B0001400035228002000090033001500E3005A
:1001C0002C0021000E0012001A0004522D00220003
:1001D0000F000C001100000050002E004A0000002B
:1001E0000100000052002E004D0000000100000040
:1001F00051002300050018000D0000004F002400EE
:1002000004003800100004522D00250016001C00C8
:100210003600E7002C0026000A00080037000352D1
:100220002800270019001B002D00E60000772A0097
:100230001D003100E500E40000002B001D0000005F
:10024000E100E00000001E001B0018002F00E2008B
:10025000007F1F0019000C0033000352280020000B
:100260000F0004003400E3002C0021000600080009
:10027000130004522D0022001A0012001C0000007E
:1002800050002E004A0000000100000052002E0025
:100290004D00000001000000510023000E00160078
:1002A000050000004F0024000B0011001000045254
:1002B0002D0025000A0015003600E7002C0026005E
:1002C0000900170037000352280027001400070018
:1002D0000D00E60000772A002D000000E500E40094
:1002E0000000010001000100010001000000010008
:1002F00001000100010001000100010001000100F6
:1003000001000100010001000100010001000100E5
:100310000100010013A715A701000100F40001006E
:100320000100010001000000F200010001000000D6
:1003300001000000F00001000100000001000000C9
:10034000F10001000100010001000000F3000100C4
:1003500042003E003A000100F500010043003F006A
:100360003B00010001000100440040003C0001008E
:1003700001000100450041003D00010001000100B5
:100380000100010001000100000000000000000069
:1003900000000000000000004B004A00290000009F
:1003A000000000002A0050002B00010000000000A7
:1003B0005200510049000000000000004C004F00B6
:1003C00028000100000000004E004D007A000000EF
:1003D000000000000000000001000000000000001C
:1003E000000000000100000000000000000000000C
:1003F0000000000000000000240021001E00010099
:1004000000000000250022001F0000000000000086
:10041000260023002000010000000000300036000C
:10042000000000000000000038003700000000005D
:10043000000016034500720067006F0044006F0063
:100440007800200045005A000000160345007200A5
:1004500067006F0044006F007800200045005A00DC
:1004600000000403090409026D00040100A0FA0958
:100470000400000103010100092111010001223FD4
:10048000000705810308000A0904010001030102B5
:1004900000092111010001224D0007058203080017
:1004A0000A090402000103000000092111010001F2
:1004B0002236000705830308000A0904030001032C
:1004C0000000000921110100012239000705840301
:1004D0001000011201100100000008EDFE071301D9
:1004E000000102000105010906A101050719E02923
:1004F000E7150025019508750181020508190129F4
:10050000059505750191029501750391010507197E
:1005100000297715002501957875018102C0050134
:100520000980A101850216010026B7001A01002AE0
:10053000B700751095018100C0050C0901A1018566
:1005400003160100269C021A01002A9C02751095D0
:10055000018100C005010902A1010901A1000509ED
:1005600019012905150025019505750181029501DF
:10057000750381010501093009311581257F950237
:100580007508810609381581257F95017508810652
:10059000050C0A38021581257F950175088106C072
:1005A000C005010906A101050719E029E715002585
:1005B00001950875018102950175088101050819E9
:1005C00001290595057501910295017503910105B4
:1005D00007190029FF150025FF950675088100C041
:1005E0000000000000000000000000010204060AF4
:1005F0000F17202C3A4A5D71879DB3C7DAE9F5FCE5
:10060000FFFCF5E9DAC7B39D87715D4A3A2C2017E4
:100610000F0A0604020100000000000000000000B4
:1006200011241FBECFEFDAE0DEBFCDBF04B603FE5C
:1006300027C08091ED019091EE01A091EF01B09162
:10064000F0018730904BA740B04BD1F41092ED01F0
:100650001092EE011092EF011092F00114BE84B7D7
:10066000877F84BF0FB6F894A89580916000886159
:1006700080936000109260000FBEE0E0FFE30995F8
:1006800011E0A0E0B1E0E8E1F7E402C005900D92CE
:10069000A433B107D9F721E0A4E3B1E001C01D9272
:1006A000AD3EB207E1F70E94BC090C948A230C947A
:1006B000000061110BC0FC018281882321F085EECE
:1006C0000E942A1003C085EE0E94F21080E090E0A4
:1006D000089508956091B1017091B2018091B301C4
:1006E0009091B4010E947A1A56985E9825982D9898
:1006F00026982E9827982F98823051F0833029F031
:10070000813049F4269A2E9A0895259A2D9A0895B3
:10071000279A2F9A089556985E9808950C946A0324
:1007200056985E9825982D9826982E9827982F9859
:100730008FEF90E0909389008093880090938B00D6
:1007400080938A0090938D0080938C00259A2D9A37
:100750002FEF80E792E0215080409040E1F700C009
:100760000000269A2E9A2FEF80E792E021508040D9
:100770009040E1F700C00000279A2F9A2FEF80E702
:1007800092E0215080409040E1F700C000002598A1
:100790002D982FEF80E792E0215080409040E1F7C4
:1007A00000C0000026982E982FEF80E792E021509D
:1007B00080409040E1F700C0000027982F9856989D
:1007C0005E9825982D9826982E9827982F9808950A
:1007D00089EA8093800089E08093810024982C9896
:1007E0003F988AB18F748AB96E98479A8BB1806BA3
:1007F0008BB9769A0E9490030C94690380E28093EF
:1008000000018091340181110EC00E944D0481E0ED
:10081000809334012FEF83ED90E32150804090408E
:10082000E1F700C0000080E40E94530480930001BF
:1008300081112EC00E947D0480930001811128C087
:100840000E947D0480930001811122C08FE30E94E9
:100850007D048093000181111BC00E94750480E417
:100860000E94530480930001811112C08CE00E9409
:100870007D048093000181110BC00E947D04809350
:100880000001811105C08FE30E947D048093000167
:100890000E9475048091000108951092B9008AE0C9
:1008A0008093B800089594EA9093BC009091BC00A6
:1008B00097FFFCCF9091B900987F983021F090314C
:1008C00011F081E008958093BB0084E88093BC0020
:1008D0008091BC0087FFFCCF8091B900887F883170
:1008E00011F0803471F780E0089584E98093BC00B2
:1008F0008091BC0084FDFCCF08958093BB0084E808
:100900008093BC008091BC0087FFFCCF9091B90020
:10091000987F81E0983209F480E0089584E880931C
:10092000BC008091BC0087FFFCCF8091BB00089584
:1009300080910001811115C080E40E9453048093CE
:10094000000181110CC082E10E947D0480930001AE
:10095000811105C08FEF0E947D04809300010E94E9
:10096000750484B1807F84B985B1807F85B98AB1EF
:10097000837F8AB98BB1837F8BB93E98469808955F
:100980000E94FE03809300010E94980480B38C7043
:1009900080BB81B3836F81BBE4E4F1E0A6E3B1E007
:1009A00011921D9281E0E235F807D1F70C94E8032B
:1009B0009F92AF92BF92CF92DF92EF92FF920F93EE
:1009C0001F93CF93DF9380910001882379F080916A
:1009D00035018F5F80933501811108C00E94FE03AD
:1009E00080930001811102C00E94900386E3E82EEB
:1009F00081E0F82E8701C0E0D0E0BB24B39492E000
:100A0000A92ECC24C394D12CC730D10500F58091F8
:100A10000001811164C080E40E94530480930001AE
:100A2000811112C082E10E947D0480930001811136
:100A30000BC0C6010C2E01C0880F0A94EAF78095FE
:100A40000E947D04809300010E94750448C0CA3052
:100A5000A1F028F4C83059F0C93061F005C0CC309D
:100A600089F070F0CD3089F0209A289810C0219A32
:100A700029980DC0229A2A980AC0239A2B9807C059
:100A8000529A01C0539A5B9802C03E9A4698E0EA97
:100A9000EA95F1F78FB181708B25799902C032E028
:100AA00001C030E0832B7C9902C034E001C030E00B
:100AB000832B7D9902C028E001C020E0822B7E9923
:100AC00002C090E101C090E0892B9FB19095991FE1
:100AD0009927991F9295990F907E892B0FC080912D
:100AE000000181114AC080E40E94530480930001F8
:100AF000882381F1912C0E947504892DD8019C9145
:100B0000981719F08C93A09201010E9498042196E5
:100B10000F5F1F4FCE30D10509F076CF80910101D4
:100B2000882369F1815080930101882339F0EFE92E
:100B3000FFE03197F1F700C0000021C0E4E4F1E0EC
:100B4000D7018D917D018193B4E4EB16B1E0FB06F2
:100B5000B9F715C083E10E947D04809300018111E3
:100B6000C9CF81E40E945304809300018111C2CF58
:100B70000E948E04982E9094BECF80E0BFCF0E943A
:100B80008E0381E0DF91CF911F910F91FF90EF9045
:100B9000DF90CF90BF90AF909F900895E82FF0E046
:100BA000EC5BFE4F8081089508958B3B910580F4A6
:100BB000883A910548F5853A9105D8F48430910535
:100BC00008F0B2C0019709F06EC081E090E008958E
:100BD000803E910508F467C0883E910508F4A4C0E2
:100BE0009C01205F31092031310508F05CC090651F
:100BF0000895853A910509F459C0863A910509F09E
:100C000058C082E890E40895883A910509F454C0E8
:100C1000893A910509F453C08A3A910509F452C002
:100C20008B3A910509F451C08C3A910509F450C0F2
:100C30008D3A910509F44FC0803B910509F44EC0EF
:100C40008E3A910509F44DC08F3A910509F44CC0D4
:100C5000813B910509F44BC0823B910509F44AC0E0
:100C6000833B910509F449C0843B910509F448C0D0
:100C7000853B910509F447C0863B910509F446C0C0
:100C8000873B910509F445C0883B910509F444C0B0
:100C9000893B910509F443C08A3B910509F442C0A0
:100CA00080E094E4089580E090E0089581E890E485
:100CB000089583E890E4089582EE94E4089589EE1F
:100CC00094E408958AEE94E4089585EB94E40895FD
:100CD00086EB94E4089587EB94E408958CEC94E417
:100CE00008958DEC94E4089583E895E408958AE8E6
:100CF00095E4089582E995E4089584E995E40895DA
:100D000081E296E4089583E296E4089584E296E40D
:100D1000089585E296E4089586E296E4089587E2D0
:100D200096E408958AE296E40895089524E5829F62
:100D3000C0011124FC0126E0729FE00DF11D112479
:100D4000E60FF11DEE0FFF1FE651FF4F85919491C5
:100D50000895880F991FFC01E05AF0408591949105
:100D60000895880F991FFC01E052FF4F85919491DF
:100D7000089524E5829FC0011124FC0146E0749F80
:100D8000E00DF11D1124E60FF11DEE0FFF1FE651DE
:100D9000FF4F859194919C013A9521154FE13407BD
:100DA00008F425C13F512115304120F49F700E9465
:100DB000B10608959C0130532115304118F499274C
:100DC000906C0895811520E5920769F40E946B14D8
:100DD0004FEF84E39CE0415080409040E1F700C039
:100DE00000000C94721B813020E5920731F4809151
:100DF000CC0181608093CC0108959C013055211570
:100E0000304108F05CC0292F33272F703327213061
:100E10003105E9F4AC0164E0440F551F6A95E1F730
:100E200044275370BC016370772702C0220F331F21
:100E30006A95E2F73C68242B352B73E0880F991FE5
:100E40007A95E1F780769927822B932B08952230AB
:100E5000310529F4982F8827816F906A08952330EF
:100E60003105A1F4AC0133E0440F551F3A95E1F789
:100E7000407E57708370992721E030E002C0220F36
:100E8000331F8A95E2F7C9019C6816C024303105EA
:100E900031F5AC0123E0440F551F2A95E1F7407E60
:100EA00057708370992721E030E002C0220F331F72
:100EB0008A95E2F7C9019A68842B952B08959C01C5
:100EC00030572115304118F49F70906208959C01AD
:100ED00030582115304118F49F70906A0895803E73
:100EE0009105E0F4803C910558F58133910509F4B2
:100EF0006FC048F48932910509F463C08A329105C4
:100F000009F46DC072C089339105E9F0823891050A
:100F1000D1F08533910509F44DC067C0833E91053A
:100F200081F138F4803E9105B9F0823E9105D9F007
:100F30005CC0863E910561F1873E9105A1F155C0E7
:100F40000E94A90608952091DE0120FD02C021FF24
:100F50004CC080EE90E049C08091DE0180FFF9CF67
:100F600089E390E042C08091DE0182FF0EC0809153
:100F7000DE0184FF03C080E090E037C083EE90E0A4
:100F800034C08091DE0182FFF2CF82EE90E02DC06E
:100F90008091DE0183FF0BC08091DE0184FDEBCFE9
:100FA00087EE90E022C08091DE0183FFF5CF86EED0
:100FB00090E01BC08091DE0185FF07C089E290E0D0
:100FC00014C08091DE0185FFF9CF85E390E00DC06C
:100FD0008091DE0186FF07C08AE290E006C0809122
:100FE000DE0186FFF9CF81E390E00E94D5050895E8
:100FF0000895809162010895CF93DF9300D01F92EE
:10100000CDB7DEB79C018091E401843019F593E0FF
:1010100099833B832A839093E9008FEF9091E800B6
:10102000815095FD06C095ED9A95F1F7000081116C
:10103000F5CF8091E80085FF0DC040E050E063E00F
:1010400070E0CE0101960E94690A8091E8008E77D7
:101050008093E8000F900F900F90DF91CF9108954B
:10106000CF93DF9300D01F92CDB7DEB72091E4017C
:10107000243021F522E029839B838A8383E08093B7
:10108000E9008FEF9091E800815095FD06C095ED45
:101090009A95F1F700008111F5CF8091E80085FF66
:1010A0000DC040E050E063E070E0CE0101960E9488
:1010B000690A8091E8008E778093E8000F900F9086
:1010C0000F90DF91CF9108959C018091E4018430CD
:1010D000F9F482E08093E9009FEF8091E80091505D
:1010E00085FD06C085ED8A95F1F700009111F5CFD9
:1010F0008091E80085FF0CC040E050E065E070E0C2
:10110000C9010E94690A8091E8008E778093E80007
:101110000895CF93DF93EC018091E401843009F0CE
:1011200046C090910C019923D9F090910D0199231B
:10113000B9F08093E9008FEF9091E800815095FD20
:1011400006C095E19A95F1F700008111F5CF8091E5
:10115000E80085FF2CC040E050E060E170E017C07F
:1011600081E08093E9008FEF9091E800815095FD38
:1011700006C095ED9A95F1F700008111F5CF8091A9
:10118000E80085FF14C040E050E068E070E0CE0168
:101190000E94690A8091E8008E778093E80080E1E0
:1011A000FE01A2E5B1E001900D928A95E1F7DF9191
:1011B000CF9108958091E301811109C00E94FA0B3B
:1011C0000E94570C8091E20084608093E2000895B1
:1011D0001092E301089508950C94A8210E94081B21
:1011E0000E94AE210E94020F0C94F80742E061ECCD
:1011F00081E00E94730B42E061EC82E00E94730B7D
:1012000042E061EC83E00E94730B42E161EC84E018
:101210000C94730B8091E601833009F455C030F4CF
:10122000813071F0823009F48EC008958A3009F45B
:101230007AC08B3009F460C0893009F09CC020C0AE
:101240008091E501813A09F096C08091E800877F9E
:101250008093E8008091E9019091EA01892B21F4C3
:1012600060E182E591E003C060E080E090E070E042
:101270000E94B40A8091E8008B778093E80008957B
:101280008091E501813209F076C08091E901909169
:10129000EA01009719F0039709F06DC08091E8000A
:1012A000877F8093E8008091E80082FD05C08091EF
:1012B000E4018111F8CF5FC08091F1008093620159
:1012C0008091E8008B7753C08091E501813A09F065
:1012D00052C08091E9019091EA01892B09F04BC03D
:1012E0008091E800877F8093E8008091E80080FF8C
:1012F000FCCF80910C0136C08091E5018132D9F597
:101300008091E9019091EA01892BA9F58091E8008B
:10131000877F8093E8000E94A80B8091E70180936B
:101320000C010C946B148091E501813221F58091C0
:10133000E800877F8093E8000E94A80B8091E80175
:101340008093630108958091E501813AA1F4809131
:10135000E800877F8093E8008091E80080FFFCCF61
:10136000809163018093F1008091E8008E778093F3
:10137000E8000C94A80B089584B7877F84BF0FB64C
:10138000F894A89580916000886180936000109225
:1013900060000FBE90E080E80FB6F8948093610083
:1013A000909361000FBE0E94510F0E94FA0B0E94A1
:1013B000570C8091E20084608093E20078940E9450
:1013C000E20E0E94530F82E091E00E94FD0E0E9407
:1013D00096218091E401853069F40E94CA1A8091B7
:1013E000E2018823B1F30E94F41A882391F30E944A
:1013F000530AEFCF0E94590FECCF292F3327233008
:101400003105C9F060F42130310581F02230310519
:1014100009F041C08DE690E026E634E040C021327C
:101420003105E1F02232310531F135C082E190E041
:1014300023ED34E034C099278130910549F028F03C
:10144000029749F5E2E3F4E005C0E2E6F4E002C009
:10145000EAE4F4E0849190E09F0121C06430D8F484
:10146000E62FF0E0EE0FFF1FEE5DFE4F2081318191
:1014700089E090E014C0643070F470E0FB01EE0F7E
:10148000FF1FE65EFE4F20813181FB01EA5EFE4FC9
:10149000808190E004C080E090E020E030E0FA013C
:1014A00031832083089580E189BD82E189BD09B43B
:1014B00000FEFDCF8091D8008F7D8093D800809171
:1014C000E00082608093E0008091E00081FDFCCF2D
:1014D0000895CF92DF92EF92FF920F931F93CF93D5
:1014E000DF93EC018B016A010E94C70B811133C0AD
:1014F000C114D10439F0F60180819181081B190BC8
:10150000C80FD91FE12CF12C0115110519F180919B
:10151000E80085FD16C08091E8008E778093E80092
:10152000C114D10449F0F60180819181E80EF91EC1
:10153000F182E08285E00FC00E94C70B882321F36F
:101540000AC089918093F10001501109FFEFEF1A51
:10155000FF0ADACF80E0DF91CF911F910F91FF90CA
:10156000EF90DF90CF9008952091EB013091EC0146
:101570002617370748F06115710539F42091E80006
:101580002E772093E80001C0B901FC0120E061152D
:10159000710579F18091E4018823F1F18530F1F151
:1015A0008091E80083FD3CC08091E80082FD2EC060
:1015B0008091E80080FFEBCF2091F3008091F20052
:1015C00090E0922B6115710551F08830910538F447
:1015D00021912093F100615071090196F3CF21E030
:1015E000089709F020E08091E8008E778093E8006A
:1015F000CECF2111CFCF0AC08091E401882361F0C2
:10160000853061F08091E80083FD0AC08091E80098
:1016100082FFF2CF80E0089582E0089583E008958C
:1016200081E008952091EB013091EC0126173707F6
:1016300048F06115710539F42091E8002E77209368
:10164000E80001C0B901FC0120E06115710591F1CC
:101650008091E401882309F440C0853009F43FC03B
:101660008091E80083FD3DC08091E80082FD2FC09D
:101670008091E80080FFE9CF2091F3008091F20093
:1016800090E0922B6115710559F08830910540F476
:1016900024912093F1003196615071090196F2CFA7
:1016A00021E0089709F020E08091E8008E77809390
:1016B000E800CBCF2111CCCF0AC08091E401882370
:1016C00061F0853061F08091E80083FD0AC080916F
:1016D000E80082FFF2CF80E0089582E0089583E081
:1016E000089581E00895982F973068F59093E90068
:1016F000981739F07091EC002091ED005091F000B6
:1017000003C0242F762F50E021FD02C09F5FECCF55
:101710003091EB003E7F3093EB003091ED003D7F48
:101720003093ED003091EB0031603093EB0070931B
:10173000EC002093ED005093F0002091EE0027FD87
:10174000E5CF80E008958F708093E90081E00895EF
:101750008091E50187FF11C08091E80082FD05C0FE
:101760008091E4018111F8CF11C08091E8008B775E
:101770000BC08091E401882349F08091E80080FF4C
:10178000F8CF8091E8008E778093E800089520914B
:10179000E4003091E50095E64091EC00842F8170E3
:1017A00040FF23C08091E80080FD1DC08091E401CE
:1017B000882399F0853099F08091EB0085FD11C068
:1017C0004091E4005091E5002417350729F391502A
:1017D00011F09A01E1CF84E0089582E0089583E05A
:1017E000089581E0089580E008954091E80042FF67
:1017F000DDCF08950E94680C0E94700CE0EEF0E0CE
:10180000808181608083E8EDF0E080818F77808344
:1018100019BCA7EDB0E08C918E7F8C9380818F7E78
:1018200080831092E30108950F931F93CF93DF936A
:101830000E94680C0E94700CC8EDD0E088818F7700
:10184000888388818068888388818F7D888319BC9C
:101850001092E4011092E0011092E2011092E10175
:1018600000EE10E0F80180818B7F808388818160A9
:10187000888342E060E080E00E94730BE1EEF0E0DC
:1018800080818E7F8083E2EEF0E0808181608083C2
:10189000808188608083F80180818E7F8083888149
:1018A00080618883DF91CF911F910F910895E8EDBA
:1018B000F0E080818F7E8083E7EDF0E080818160C1
:1018C000808384E082BF81E08093E3010C94140C58
:1018D000E8EDF0E080818E7F80831092E200089531
:1018E0001092DA001092E10008951F920F920FB645
:1018F0000F9211242F933F934F935F936F937F9396
:101900008F939F93AF93BF93EF93FF938091E100E9
:1019100082FF0BC08091E20082FF07C08091E1004E
:101920008B7F8093E1000E94E10E8091DA0080FFBE
:101930001FC08091D80080FF1BC08091DA008E7F8D
:101940008093DA008091D90080FF0DC080E189BDCD
:1019500082E189BD09B400FEFDCF81E08093E401FE
:101960000E94DA0805C019BC1092E4010E94E80840
:101970008091E10080FF19C08091E20080FF15C0D6
:101980008091E2008E7F8093E2008091E20080618E
:101990008093E2008091D80080628093D80019BCC7
:1019A00085E08093E4010E94EC088091E10084FFCF
:1019B00030C08091E20084FF2CC080E189BD82E1CB
:1019C00089BD09B400FEFDCF8091D8008F7D809342
:1019D000D8008091E1008F7E8093E1008091E20049
:1019E0008F7E8093E2008091E20081608093E2002C
:1019F0008091E001882311F084E007C08091E3002A
:101A000087FD02C081E001C083E08093E4010E9471
:101A1000EE088091E10083FF29C08091E20083FFFE
:101A200025C08091E100877F8093E10082E0809370
:101A3000E4011092E0018091E1008E7F8093E1004B
:101A40008091E2008E7F8093E2008091E2008061CD
:101A50008093E20042E060E080E00E94730B80919E
:101A6000F00088608093F0000E94EB08FF91EF91F6
:101A7000BF91AF919F918F917F916F915F914F91A6
:101A80003F912F910F900FBE0F901F9018951F92AE
:101A90000F920FB60F9211242F933F934F935F93A2
:101AA0006F937F938F939F93AF93BF93CF93DF9366
:101AB000EF93FF93C091E900CF708091EC00D82F95
:101AC000D17080FDD0E81092E9008091F000877F0E
:101AD0008093F00078940E948B0D1092E900809121
:101AE000F00088608093F000CD2BCF70C093E900A8
:101AF000FF91EF91DF91CF91BF91AF919F918F9126
:101B00007F916F915F914F913F912F910F900FBEF9
:101B10000F901F9018951F93CF93DF93CDB7DEB72B
:101B2000AA970FB6F894DEBF0FBECDBFE5EEF1E089
:101B30008091F100819321E0ED3EF207C9F70E9408
:101B40000A098091E80083FF24C18091E50190910A
:101B5000E601492F50E04A30510508F01AC1FA0158
:101B6000EA5AFF4F0C943F23803881F0823809F005
:101B700010C18091E9018F708093E9008091EB00A2
:101B800085FB882780F91092E90006C08091E10169
:101B90009091E201911182609091E800977F90937B
:101BA000E8008093F1001092F100C8C0282F2D7F2B
:101BB00009F0EFC0882319F0823061F0EAC080910B
:101BC000E701813009F0E5C0933009F080E08093AF
:101BD000E2012BC08091E701811127C08091E901CA
:101BE0008F7009F4D6C08093E9002091EB0020FFAC
:101BF0001CC0933021F48091EB00806214C090915E
:101C0000EB0090619093EB0021E030E0A90102C06D
:101C1000440F551F8A95E2F74093EA001092EA00BC
:101C20008091EB0088608093EB001092E900809136
:101C3000E800877F86C08111ACC01091E7011F7753
:101C40008091E3008078812B8093E3008091E8000D
:101C5000877F8093E8000E94A80B8091E80080FFB6
:101C6000FCCF8091E30080688093E300111102C0F3
:101C700082E001C083E08093E4018BC08058823011
:101C800008F087C08091E7019091E8018C3D53E016
:101C9000950779F583E08A838AE289834FB7F894C0
:101CA000DE01139620E03EE051E2E32FF0E0509396
:101CB0005700E49120FF03C0E295EF703F5FEF70A3
:101CC0008E2F90E0EA3010F0C79601C0C0968D9339
:101CD0009D932F5F243149F74FBF8091E800877FA4
:101CE0008093E8006AE270E0CE0101960E94B40A97
:101CF00014C0AE014F5F5F4F6091E9010E94FD0982
:101D0000BC01892B09F445C09091E800977F90931E
:101D1000E80089819A810E94120B8091E8008B77FC
:101D20008093E80036C08038A1F58091E800877F75
:101D30008093E8008091E0018093F1008091E800B9
:101D40008E778093E8000E94A80B23C0811121C0E8
:101D50008091E7019091E80199270297D4F480914E
:101D6000E800877F8093E8008091E7018093E0019D
:101D70000E94A80B8091E001811106C08091E300D0
:101D800087FD02C081E001C084E08093E4010E94ED
:101D9000F6088091E80083FF0AC08091E800877F01
:101DA0008093E8008091EB0080628093EB00AA961C
:101DB0000FB6F894DEBF0FBECDBFDF91CF911F915C
:101DC00008950895CF938091E4018823A1F0C091F4
:101DD000E900CF709091EC00892F817090FD80E830
:101DE000C82B1092E9008091E80083FD0E948B0DC2
:101DF000CF70C093E900CF910895909369018093CB
:101E000068010895E0916801F0916901309721F02F
:101E10000190F081E02D099480E00895E09168013F
:101E2000F0916901309721F00280F381E02D09944F
:101E30000895E0916801F0916901309721F00480E4
:101E4000F581E02D09940895209166013091670194
:101E50002817390771F09093670180936601E0912C
:101E60006801F0916901309721F00680F781E02D3B
:101E7000099408952091640130916501281739076C
:101E800071F09093650180936401E0916801F09195
:101E90006901309721F00084F185E02D09940895BF
:101EA00008950C94500F0E940E1B0E94C0040C94C5
:101EB000D41BCF92DF92EF92FF920F931F93CF9399
:101EC000DF93CDB7DEB72B970FB6F894DEBF0FBE0A
:101ED000CDBF0E94D8048BE6C82E81E0D82E00E04A
:101EE00010E0E02E802F0E94CE05F60141916F0197
:101EF000F82EF426B1F40F5F1F4F0E30110589F74D
:101F00008FEF89838A831B820E94171B8160782F41
:101F10009D838C8349815A816B818D810E94FC0F46
:101F200040C09091CC0191FF04C08B870E94D405E2
:101F30008B8520E030E04F2D50E0922FBA01022E29
:101F400002C0759567950A94E2F760FF24C02E835E
:101F5000EF8221E030E0690102C0CC0CDD1C9A95D3
:101F6000E2F790E08C219D21892B09F420E028875D
:101F70000E94171B8160782F9A8789874E815F8125
:101F800068858A850E94FC0FF801E559FE4F808123
:101F9000C826C08206C02F5F3F4F2630310569F644
:101FA000AACF0E94BB1E0E94020F90916A0189175E
:101FB000A1F00E94020F80936A012B960FB6F8944D
:101FC000DEBF0FBECDBFDF91CF911F910F91FF906C
:101FD000EF90DF90CF900C94F8072B960FB6F89403
:101FE000DEBF0FBECDBFDF91CF911F910F91FF904C
:101FF000EF90DF90CF900895CF93DF93CDB7DEB70A
:102000002B970FB6F894DEBF0FBECDBF4F83588716
:1020100069877A878B87DE01119686E0FD01119230
:102020008A95E9F785E0FE01379601900D928A9531
:10203000E1F749815A816B817C818D819E810E946B
:10204000FF162B960FB6F894DEBF0FBECDBFDF9103
:10205000CF910895CF93C82F882309F4C1C0823847
:1020600059F40E94020F81FDBBC089E30E949C19B4
:102070000E94541A89E30CC0833879F40E94020F3D
:1020800080FDAEC083E50E949C190E94541A83E52E
:102090000E94DB19CF910C94541A843859F40E9491
:1020A000020F82FD9DC087E40E949C190E94541A71
:1020B00087E4EECF8CEF8C0F813A48F48C2F0E948E
:1020C000FB2081118DC08C2F0E949C19E3CF80E2F0
:1020D0008C0F883048F4C77081E001C0880FCA9522
:1020E000EAF70E941D1AD6CF8BE58C0F833078F467
:1020F000C53A29F0C63A31F083E890E005C081E89E
:1021000090E002C082E890E0CF910C94240F88E523
:102110008C0F833108F064C0C83A39F1C93A41F1F3
:10212000CA3A49F1CB3A51F1CC3A59F1CD3A61F181
:10213000C03B69F1CE3A71F1CF3A79F1C13B81F1FF
:10214000C23B89F1C33B91F1C43B99F1C53BA1F17D
:10215000C63BA9F1C73BB1F1C83BB9F1C93BC1F1DD
:10216000CA3BC9F180E090E038C082EE90E035C013
:1021700089EE90E032C08AEE90E02FC085EB90E0CF
:102180002CC086EB90E029C087EB90E026C08CEC59
:1021900090E023C08DEC90E020C083E891E01DC06A
:1021A0008AE891E01AC082E991E017C084E991E0E1
:1021B00014C081E292E011C083E292E00EC084E29A
:1021C00092E00BC085E292E008C086E292E005C092
:1021D00087E292E002C08AE292E0CF910C943A0F3B
:1021E000CF910895882309F44BC0823859F40E9496
:1021F000020F81FF45C089E30E949C190E94541A76
:1022000089E30CC0833871F40E94020F80FF38C04C
:1022100083E50E949C190E94541A83E50E94DB19F1
:102220000C94541A843859F40E94020F82FF28C07B
:1022300087E40E949C190E94541A87E4EFCF9CEF18
:10224000980F913A58F390E2980F983050F48770B5
:1022500091E001C0990F8A95EAF7892F0E94231A0D
:10226000DFCF9BE5980F933020F480E090E00C9452
:10227000240F885A833120F480E090E00C943A0FC8
:102280000895882321F00E941D1A0C94541A089571
:10229000882321F00E94231A0C94541A0895BF92A7
:1022A000CF92DF92EF92FF920F931F93CF93DF9322
:1022B00000D000D000D0CDB7DEB77C0185E0F701BB
:1022C000DE01119601900D928A95E1F7F701838165
:1022D0009481892B09F4DDC2908181818F3F19F4AB
:1022E0009F3F09F4D6C2F7010281258122952F7004
:1022F00099838A8389819A812E830E945B19182F82
:10230000B92E0E945A190E942118EB2DE295EF7008
:102310004E2F50E0FA01E05AFF4F2E810C943F23DC
:102320008B2D807F9B2D9F70F92E882319F0F294BE
:1023300080EFF822002349F0FF2009F457C28F2DC7
:102340000E942D1A0E94541A51C2812F0E94F2102D
:10235000FF2009F49EC28F2D0E94331A26960FB6D5
:10236000F894DEBF0FBECDBFDF91CF911F910F91CB
:10237000FF90EF90DF90CF90BF900C94541A3B2DBC
:10238000307F8B2D8F70303211F08295807F11233A
:1023900019F0113021F12CC00023B9F0222309F4E7
:1023A00090C1213009F08DC126960FB6F894DEBF9A
:1023B0000FBECDBFDF91CF911F910F91FF90EF9096
:1023C000DF90CF90BF900C943D1A222319F021305A
:1023D00009F45FC28E830E94401A8E8186C1002359
:1023E00021F0223008F055C26CC1211152C27DC1CA
:1023F000002321F0222309F464C1F8C1222309F447
:1024000074C109C28B2D86958695837019F0813031
:10241000D1F03FC2002321F0812F9B2D937002C089
:1024200080E090E026960FB6F894DEBF0FBECDBFD9
:10243000DF91CF911F910F91FF90EF90DF90CF90A0
:10244000BF900C94240F002321F0812F9B2D9370BB
:1024500002C080E090E026960FB6F894DEBF0FBE73
:10246000CDBFDF91CF911F910F91FF90EF90DF9043
:10247000CF90BF900C943A0F812F002319F00E9447
:10248000C31D02C00E942B1E26960FB6F894DEBF15
:102490000FBECDBFDF91CF911F910F91FF90EF90B5
:1024A000DF90CF90BF900C94B01E8B2D837009F0FD
:1024B00075C00111EEC1812F829586958770880FB6
:1024C000880F912F9F70C92ED12CE12CF12C082E52
:1024D00004C0CC0CDD1CEE1CFF1C0A94D2F714FFC8
:1024E00012C00FE010E020E030E004C0000F111F28
:1024F000221F331F8A95D2F7C901B80160957095E4
:102500008095909503C060E070E0CB014B2D46951F
:10251000469543704230C1F060F56C297D298E29C3
:102520009F29413051F126960FB6F894DEBF0FBEB9
:10253000CDBFDF91CF911F910F91FF90EF90DF9072
:10254000CF90BF900C9448186C297D298E299F2923
:1025500026960FB6F894DEBF0FBECDBFDF91CF91A8
:102560001F910F91FF90EF90DF90CF90BF900C9450
:1025700064180E944818C701B60126960FB6F89451
:10258000DEBF0FBECDBFDF91CF911F910F91FF90A6
:10259000EF90DF90CF90BF900C942C18002319F08F
:1025A0008B2D817001C08695882309F472C1812F1B
:1025B000829586958770880F880F912F9F70C92EFE
:1025C000D12CE12CF12C082E04C0CC0CDD1CEE1C0F
:1025D000FF1C0A94D2F714FF12C00FE010E020E0B5
:1025E00030E004C0000F111F221F331F8A95D2F75D
:1025F000C901B801609570958095909503C060E021
:1026000070E0CB014B2D4695469543704230C1F0AA
:1026100060F56C297D298E299F29413051F126963C
:102620000FB6F894DEBF0FBECDBFDF91CF911F91E3
:102630000F91FF90EF90DF90CF90BF900C942219F4
:102640006C297D298E299F2926960FB6F894DEBF26
:102650000FBECDBFDF91CF911F910F91FF90EF90F3
:10266000DF90CF90BF900C943E190E942219C701B1
:10267000B60126960FB6F894DEBF0FBECDBFDF9130
:10268000CF911F910F91FF90EF90DF90CF90BF906F
:102690000C940619103FD1F118F4103E50F4A1C06B
:1026A000123F09F463C008F44CC0133F09F473C02F
:1026B00098C01F708B2D8F710023A1F00E949F186E
:1026C000812F26960FB6F894DEBF0FBECDBFDF91E7
:1026D000CF911F910F91FF90EF90DF90CF90BF901F
:1026E0000C9441110E94C018812F26960FB6F894C1
:1026F000DEBF0FBECDBFDF91CF911F910F91FF9035
:10270000EF90DF90CF90BF900C9448110023A9F078
:102710002111BFC08B2D8F7126960FB6F894DEBFA6
:102720000FBECDBFDF91CF911F910F91FF90EF9022
:10273000DF90CF90BF900C94E518223008F0A9C02C
:10274000E9CF0023A9F08B2D8F7126960FB6F89450
:10275000DEBF0FBECDBFDF91CF911F910F91FF90D4
:10276000EF90DF90CF90BF900C949F18002359F307
:102770008B2D8F7126960FB6F894DEBF0FBECDBF9E
:10278000DF91CF911F910F91FF90EF90DF90CF904D
:10279000BF900C94C018002399F08B2D8F71269652
:1027A0000FB6F894DEBF0FBECDBFDF91CF911F9162
:1027B0000F91FF90EF90DF90CF90BF900C948A180C
:1027C00026960FB6F894DEBF0FBECDBFDF91CF9136
:1027D0001F910F91FF90EF90DF90CF90BF900C94DE
:1027E00080180023A9F0222309F4ADCF812F26966B
:1027F0000FB6F894DEBF0FBECDBFDF91CF911F9112
:102800000F91FF90EF90DF90CF90BF900C942A1023
:10281000222309F4ADCF812F26960FB6F894DEBFA0
:102820000FBECDBFDF91CF911F910F91FF90EF9021
:10283000DF90CF90BF900C94F2104B2D4F70612F12
:10284000C7010E94590326960FB6F894DEBF0FBE4B
:10285000CDBFDF91CF911F910F91FF90EF90DF904F
:10286000CF90BF900C94A4174B2D4F70612FC701D0
:1028700026960FB6F894DEBF0FBECDBFDF91CF9185
:102880001F910F91FF90EF90DF90CF90BF900C942D
:10289000950626960FB6F894DEBF0FBECDBFDF912A
:1028A000CF911F910F91FF90EF90DF90CF90BF904D
:1028B00008950E943A1A0E940F1A0E94541A0E9408
:1028C000601F0E94B01E80E090E00E94240F80E014
:1028D00090E00C943A0F0E942A1A0C9459140E940A
:1028E0005B19292F22952F702C3030F42A3048F4B0
:1028F0002250223078F405C02C3041F02F3031F0D6
:1029000009C0803E48F0803F29F406C093FB882729
:1029100080F9089580E0089581E00895CF93DF93D2
:1029200000D000D01F92CDB7DEB70F900F900F9060
:102930000F900F90DF91CF910895CF93DF9300D048
:1029400000D000D0CDB7DEB726960FB6F894DEBF24
:102950000FBECDBFDF91CF9108951F93CF93DF932B
:10296000C091790116E080917A01C81799F0D0E002
:102970001C9FF0011D9FF00D1124E558FE4F408172
:10298000518162817381848195810E949D14219679
:10299000C770E9CFDF91CF911F9108954091AB01AE
:1029A0005091AC016091AD017091AE018091AF0189
:1029B0009091B0010C949D148091B00182958F701C
:1029C00009F054C08091AD01882309F44FC0809173
:1029D0007901A0917A014091AE015091AF016091CF
:1029E000AB017091AC01B6E08A1709F43FC090E0EA
:1029F00041155105C1F17F3F11F46F3FA1F1B89F1F
:102A0000F001B99FF00D1124E558FE4F21812713E5
:102A10002AC02081261327C02281211124C02381AE
:102A200034812417350710F421503109241B350B4C
:102A3000283C3105C0F42091B0012F702061209313
:102A4000B00126E0289FF001299FF00D1124E058E5
:102A5000FE4F80818F70806180838BEA91E00E94BD
:102A60004F110C94AD1401968770BECF0895CF928C
:102A7000DF92EF92FF920F931F93CF93DF93CDB727
:102A8000DEB762970FB6F894DEBF0FBECDBF8C01E4
:102A900085E0F801DE011D9601900D928A95E1F71F
:102AA000D8014C9111965C91119712966C9180917E
:102AB000AE019091AF01009709F475C13091AB015F
:102AC0007091AC017F3F19F43F3F09F46CC1F801EC
:102AD000C380D480E090AD01EE2009F4BEC0209107
:102AE000B001C816D90628F0D601A81BB90BCD0134
:102AF00004C0809590958C0D9D1DFF24F394883C17
:102B0000910578F0F12C207F09F0C4C07C2DD98A82
:102B1000C88A89890E948E148BEA91E00E944F1125
:102B2000AFC0822F807F09F045C0571313C04313F5
:102B300011C061110FC02F7020612093B0010E945D
:102B4000CE148BEA91E00E944F118091B001F80100
:102B500085832EC0CD2819F15F3F11F44F3FF9F066
:102B6000F62E61111CC08091790120917A0136E026
:102B7000821709F45BC090E0389FF001399FF00D97
:102B80001124E558FE4F7181571306C07081471319
:102B900003C07281711103C001968770E9CFF62ED0
:102BA000662309F41CC18091B00181608093B0015B
:102BB000F12C15C1571309C0431307C0611105C09B
:102BC0008091B001F8018583C8C04D875E878D85EF
:102BD0009E856A8B0E946F146A898823D1F16623CF
:102BE000C1F12091B001822F82958F7090E0029701
:102BF00074F08091AB019091AC0198878F83198616
:102C0000DB86CA862C87CE0107960E944F1186E08C
:102C1000F801ABEAB1E001900D928A95E1F70E94CC
:102C2000DC140E94CE14FF24F394D9C04D875E8734
:102C30008D859E850E945B19292F22952F70223049
:102C400008F0C1C09F7009F0BBC0805E883008F4F6
:102C5000C6C0C8010E944F11E6CFC816D90608F4B5
:102C600053C0F601E81BF90BCF01883C910508F42D
:102C700050C0F12C7C2DD98AC88A89890E948E1473
:102C8000EBEAF1E086E0DF011D928A95E9F70E9408
:102C9000CE14A5C0571314C0431312C0611110C045
:102CA0008091B001F8018583C8010E944F1186E030
:102CB000EBEAF1E0DF011D928A95E9F7FE2C8FC067
:102CC0004D875E878D859E856A8B0E946F146A8909
:102CD000882309F4BECF662309F4BBCF2091B0014D
:102CE000822F82958F7090E002970CF490CF8091A4
:102CF000AB019091AC019A8389831B82DD82CC82E7
:102D00002E83CE01019681CF809590958C0D9D1DCF
:102D1000ACCFF62E662309F49CCF571333C0431370
:102D200031C02091B00120FD24C0822F82958F7088
:102D3000482F50E041155105E1F0D80115962C932C
:102D400015974F30510549F08F5F982F9295907FDE
:102D5000822F8F70892B15968C93C8010E944F117A
:102D600086E0F801ABEAB1E001900D928A95E1F7B7
:102D70008ECF86E0F801ABEAB1E001900D928A9522
:102D8000E1F72DC04D875E878D859E850E946F146B
:102D900081113DCF8091B00181608093B001C80165
:102DA0000E944F111CC0662309F453CF4D875E87E4
:102DB0008D859E850E946F14882309F44ACF27CF02
:102DC000811143CF0CC0243008F043CF9F7009F429
:102DD0003CCFD80115969C91907F09F036CF8F2D6E
:102DE00062960FB6F894DEBF0FBECDBFDF91CF91D4
:102DF0001F910F91FF90EF90DF90CF9008951F9358
:102E0000CF93DF93CDB7DEB72C970FB6F894DEBF24
:102E10000FBECDBF4F83588769877A878B879C8782
:102E2000CE0107960E943715882371F08A859B850D
:102E3000892B09F441C088858F3F09F065C08F81D7
:102E40008F3F09F061C038C086E0FE013796DE0191
:102E5000119601900D928A95E1F76A857B8561153F
:102E6000710551F1FF81E885EF3F11F4FF3F21F13A
:102E700020917A0130E0C90101968770992740912D
:102E8000790150E08417950709F447C0F983EA8374
:102E90007D836C8396E0929FD001939FB00D1124A7
:102EA000A558BE4FFE01319601900D929A95E1F71B
:102EB00080937A010E94AD1416E08091790190917F
:102EC0007A018917B9F1189FC001112485589E4FC6
:102ED0000E943715882371F1E09179011E9FF0015E
:102EE0001124E558FE4F40815181628173818481B4
:102EF00095810E949D148091790190E001968770E0
:102F0000992780937901D9CF4F81588569857A8532
:102F10008B859C850E949D14CFCF0E946B141092CC
:102F20007A0110927901EBEAF1E086E0DF011D926F
:102F30008A95E9F72C960FB6F894DEBF0FBECDBF89
:102F4000DF91CF911F910895EF92FF920F931F93FE
:102F5000CF93DF938C01892B09F46CC0F12CEE2404
:102F6000E394E8012196F8018491843740F4843099
:102F700008F051C0813081F0823019F15BC0853793
:102F800009F444C0A8F19CE7980F903708F052C0AC
:102F90008F770E94F21041C00E5F1F4FFE01849197
:102FA00090E2980F983050F48770FE2D01C0FF0F0B
:102FB0008A95EAF78F2F0E942D1A14C00E942A10BA
:102FC0002DC00E5F1F4FFE01849190E2980F983044
:102FD00060F48770FE2D01C0FF0F8A95EAF78F2FEE
:102FE0000E94331A0E94541A19C00E94F21016C08F
:102FF0000E5F1F4FFE01C491CC2381F08FE99FE04B
:103000000197F1F700C00000C150F6CF0E5F1F4FCF
:10301000FE01F49003C00E942A108E018F2D882398
:1030200009F49FCFEFE9FFE03197F1F700C000000E
:103030008150F5CFDF91CF911F910F91FF90EF90CD
:10304000089508956093B5017093B6018093B70118
:103050009093B8010C9459140F931F930091B501EC
:103060001091B6012091B7013091B801DC01CB017C
:10307000802B912BA22BB32B8093B5019093B6019B
:10308000A093B701B093B8011F910F910C945914FC
:103090000F931F930091B5011091B6012091B701D4
:1030A0003091B801DC01CB0180239123A223B3230B
:1030B0008093B5019093B601A093B701B093B80186
:1030C0001F910F910C9459140F931F930091B50108
:1030D0001091B6012091B7013091B801DC01CB010C
:1030E00080279127A227B3278093B5019093B6013B
:1030F000A093B701B093B8011F910F910C9459148C
:103100001092B1011092B2011092B3011092B40169
:103110000C94591441E050E060E070E004C0440FAA
:10312000551F661F771F8A95D2F74093B1015093C0
:10313000B2016093B3017093B4010C94591441E04F
:1031400050E060E070E004C0440F551F661F771F19
:103150008A95D2F78091B1019091B201A091B3010B
:10316000B091B401482B592B6A2B7B2B4093B101B2
:103170005093B2016093B3017093B4010C9459144D
:1031800041E050E060E070E004C0440F551F661F4E
:10319000771F8A95D2F740955095609570958091EC
:1031A000B1019091B201A091B301B091B401482353
:1031B00059236A237B234093B1015093B20160935A
:1031C000B3017093B4010C94591441E050E060E0F5
:1031D00070E004C0440F551F661F771F8A95D2F711
:1031E0008091B1019091B201A091B301B091B4016D
:1031F000482759276A277B274093B1015093B20192
:103200006093B3017093B4010C9459140F931F93FE
:103210000091B1011091B2012091B3013091B4013C
:10322000DC01CB01802B912BA22BB32B8093B1011E
:103230009093B201A093B301B093B4011F910F9189
:103240000C9459140F931F930091B1011091B20186
:103250002091B3013091B401DC01CB018023912393
:10326000A223B3238093B1019093B201A093B30141
:10327000B093B4011F910F910C9459140F931F93A5
:103280000091B1011091B2012091B3013091B401CC
:10329000DC01CB0180279127A227B3278093B101BE
:1032A0009093B201A093B301B093B4011F910F9119
:1032B0000C9459140895CF92DF92EF92FF920F93DE
:1032C0001F93CF93DF938C01C090B101D090B201D6
:1032D000E090B301F090B4018091B5019091B601F6
:1032E000A091B701B091B801C82AD92AEA2AFB2ACD
:1032F000CFE1D0E0D701C6010C2E04C0B695A7954A
:10330000979587950A94D2F780FF07C0B8018C2F54
:103310000E94B9068130910531F4219758F7B80120
:1033200080E00E94B906DF91CF911F910F91FF902D
:10333000EF90DF90CF90089590910C019923F1F0D8
:1033400090910D019923D1F0982F96959695969589
:103350009F3080F5E0910E01F0910F01E90FF11D12
:10336000877021E030E0A90102C0440F551F8A9503
:10337000E2F7CA019181892B8183089520910E0182
:1033800030910F01F90132969FEF40E0519185177E
:1033900089F09F3F19F4511101C0942F4F5F4E30B7
:1033A000A9F79F3F39F0F901E90FF11D97FDFA9553
:1033B00082830895089590910C019923F9F09091DA
:1033C0000D019923D9F0982F9695969596959F3053
:1033D00028F5E0910E01F0910F01E90FF11D8770C2
:1033E00021E030E0A90102C0440F551F8A95E2F7A1
:1033F000CA018095918189238183089520910E01CE
:1034000030910F01F9013296205F3F4F908189136F
:1034100001C010823196E217F307C1F7089581E0E9
:1034200090E0E0910E01F0910F01E80FF91F10827A
:10343000019680319105A9F708959091CB01892BD0
:103440008093CB01089580959091CB01892380933F
:10345000CB0108951092CB0108959091CA01892B58
:103460008093CA01089580959091CA018923809321
:10347000CA0108951092CA0108958093B901089570
:103480001092B901089580910E0190910F01FC01F5
:1034900031969C01205F3F4F80E0919191118F5FA9
:1034A000E217F307D1F70895E0910E01F0910F01B3
:1034B0008091CB018083E0910E01F0910F0190810A
:1034C0008091CA01892B80838091B901882361F0A2
:1034D000E0910E01F0910F019081892B80830E9471
:1034E000431A81111092B90180910E0190910F0140
:1034F0000C940E0FCF92DF92EF92FF926C01EE24AC
:10350000FF24C114D104E104F10421F0C701B60184
:1035100020E101C020E0C72ED82EE92EFF24C114DF
:10352000D104E104F10419F0285FC701B6016B0171
:103530007C0154E0F694E794D794C7945A95D1F758
:10354000C114D104E104F10419F02C5FC701B601E4
:103550006B017C0142E0F694E794D794C7944A95B6
:10356000D1F7C114D104E104F10419F02E5FC701B1
:10357000B601DC01CB01B695A79597958795892B68
:103580008A2B8B2B09F02F5F822FFF90EF90DF901B
:10359000CF9008958091E401843011F120E488E116
:1035A00090E00FB6F894A895809360000FBE20932A
:1035B000600083B7817F846083BF83B7816083BFEE
:1035C0007894889583B78E7F83BF0FB6F894A895BB
:1035D00080916000886180936000109260000FBE4F
:1035E000089508950C94F11ACF930E94F21A0E9444
:1035F000D8040E94F11AC0E08C2F0E94CE058111E0
:1036000004C0CF5FCE30C1F701C081E0CF910895F3
:103610000E946B140E94020F0C94F80782E084BD94
:1036200093E095BD9AEF97BD80936E0008952FB7F4
:10363000F8948091CD019091CE01A091CF01B091ED
:10364000D0012FBF0895CF92DF92EF92FF920F9398
:103650001F932FB7F8944091CD015091CE01609106
:10366000CF017091D0012FBF6A017B01EE24FF24AE
:103670008C0120E030E0C016D106E206F30610F41B
:10368000415051099A01281B390BC9011F910F9113
:10369000FF90EF90DF90CF9008951F920F920FB69A
:1036A0000F9211248F939F93AF93BF938091CD017D
:1036B0009091CE01A091CF01B091D0010196A11DB2
:1036C000B11D8093CD019093CE01A093CF01B09313
:1036D000D001BF91AF919F918F910F900FBE0F902E
:1036E0001F9018950E94FA0BF8942FEF87EA91E645
:1036F000215080409040E1F700C0000087E090EB4F
:10370000DC018093ED019093EE01A093EF01B09363
:10371000F0019CE088E10FB6F894A89580936000D2
:103720000FBE90936000FFCFEF92FF920F931F9315
:10373000CF93DF93D82FC0E08C2F0E94CE0500E0FE
:1037400010E0E82EF12CC701002E02C09595879558
:103750000A94E2F780FD06C00F5F1F4F0630110587
:1037600091F709C0602F7C2F80E00E9496068D1390
:10377000F3CF81E004C0CF5FCE30F1F680E0DF917F
:10378000CF911F910F91FF90EF900895CF93C82F85
:103790008CE20E94941B882321F08C2FCF910C94F3
:1037A000941B80E0CF910895CF930E941B1D81113F
:1037B00002C00E94011DC5E6C15049F00E94D80414
:1037C0008FE39CE90197F1F700C00000F5CF89E293
:1037D0000E94C61B811113C18AE20E94C61B81117F
:1037E0000E94011D85E00E94C61B81110E94721B70
:1037F0000E94261D8093CC0187E00E94C61B88236F
:10380000A9F18BE10E94C61B882351F08091CC0165
:1038100081FB222720F991E0922790FB81F90EC0CD
:103820008EE00E94C61B882361F08091CC0182FB50
:10383000222720F991E0922790FB82F98093CC0116
:1038400015C080E10E94C61B9091CC01882341F0F5
:1038500093FB222720F981E0822780FB93F904C0A3
:10386000892F809580FB90F99093CC018091CC01B9
:103870000E942A1D0E94381D8093DE0180EE0E9466
:10388000C61B882341F08091DE01982F909590FB14
:1038900080F98093DE0189E30E94C61B882359F0DA
:1038A0008091DE0181FB222720F991E0922790FB95
:1038B00081F98093DE0182EE0E94C61B882359F0B5
:1038C0008091DE0182FB222720F991E0922790FB74
:1038D00082F98093DE0186EE0E94C61B882359F090
:1038E0008091DE0183FB222720F991E0922790FB53
:1038F00083F98093DE0183EE0E94C61B882359F072
:103900008091DE0184FB222720F991E0922790FB31
:1039100084F98093DE0185E30E94C61B882359F059
:103920008091DE0185FB222720F991E0922790FB10
:1039300085F98093DE0181E30E94C61B882359F03C
:103940008091DE0186FB222720F991E0922790FBEF
:1039500086F98093DE0181E10E94C61B882359F01D
:103960008091DE0187FB222720F991E0922790FBCE
:1039700087F98093DE018091DE010E943C1D8091D9
:10398000DE0187FB882780F980930D0187E20E9482
:10399000C61BC82F8EE10E94C61B8111C2608FE139
:1039A0000E94C61B8111C46080E20E94C61B811167
:1039B000C86081E20E94C61B8111C06182E20E9440
:1039C000C61B8111C06283E20E94C61B8111C064C4
:1039D00084E20E94C61B882311F0C06802C0CC2379
:1039E00029F08C2F0E94331D6C2F03C00E942F1DC5
:1039F000682F70E080E090E0CF910C942218CF9176
:103A000008956DEE7EEF80E090E00E94752360E007
:103A100082E090E00E94672360E083E090E00E94F3
:103A2000672360E084E090E00E94672360E085E027
:103A300090E00C94672380E090E00E94612321E0F5
:103A40008D3E9E4F09F020E0822F089582E090E0A5
:103A50000C945923682F82E090E00C94672383E054
:103A600090E00C945923682F83E090E00C94672336
:103A700084E090E00C945923682F84E090E00C944B
:103A800067238091D30180FF0BC06091130185E013
:103A9000689FB001112475956795759567952BC042
:103AA00081FF09C06091130185E0689FB001112476
:103AB0007595679520C082FF07C06091130185E06E
:103AC000689FB001112417C09091D4019923D1F0BF
:103AD00060911201961788F72091130185E0289FC5
:103AE00090011124929FA001939F500D112470E02A
:103AF000CA010E942B236038710540F461157105DD
:103B000019F406C065E070E0862F08958FE70895E8
:103B100081E008958091D30180FF08C06091110178
:103B200070E0759567957595679521C081FF06C012
:103B30006091110170E07595679519C082FF04C00E
:103B40006091110170E010C09091D401992399F017
:103B5000609110019617A0F780911101899FC00113
:103B6000112470E00E942B236038710540F4611528
:103B7000710519F406C061E070E0862F08958FE7A3
:103B8000089581E00895803F21F40E94411D8195B0
:103B900004C0813F29F40E94411D8093D7010895FC
:103BA000823F21F40E94411D819504C0833F29F486
:103BB0000E94411D8093D6010895893F19F40E9407
:103BC0008A1D05C08A3F31F40E948A1D8195809329
:103BD000D80108958B3F21F40E948A1D819504C06D
:103BE0008C3F29F40E948A1D8093D9010895843F57
:103BF00021F48091D501816017C0853F21F4809127
:103C0000D501826011C0863F21F48091D501846086
:103C10000BC0873F21F48091D501886005C0883FA3
:103C200031F48091D50180618093D50108958D3F55
:103C300021F48091D30181600BC08E3F21F48091EB
:103C4000D301826005C08F3F29F48091D301846045
:103C50008093D3010895803F39F48091D70187FF85
:103C60006CC01092D70169C0813F29F48091D701BF
:103C70001816BCF362C09091D601823F29F497FFD9
:103C80005CC01092D60159C0833F19F41916CCF3C9
:103C900054C0893F41F48091D80118160CF04DC0F2
:103CA0001092D8014AC08A3F29F48091D80187FF39
:103CB00044C0F6CF8B3F39F48091D90187FF3DC0D6
:103CC0001092D9013AC08C3F29F48091D90118167D
:103CD000BCF333C0843F21F48091D5018E7F17C09F
:103CE000853F21F48091D5018D7F11C0863F21F45D
:103CF0008091D5018B7F0BC0873F21F48091D50146
:103D0000877F05C0883F31F48091D5018F7E8093F5
:103D1000D50113C08D3F21F48091D3018E7F0BC05C
:103D20008E3F21F48091D3018D7F05C08F3F29F410
:103D30008091D3018B7F8093D3018091D601811133
:103D40000EC08091D70181110AC08091D8018111E4
:103D500006C08091D901811102C01092D40108954A
:103D600085ED91E00E94190F0E94171B9093D201DC
:103D70008093D10108951F93CF93DF938091D10158
:103D80009091D2010E94231BAC019091D401992300
:103D900021F02091140130E006C0209115018AE045
:103DA000289F900111244217530708F485C0809181
:103DB000D601C091D701D091D8011091D9018111BC
:103DC00007C0C11175C0D11173C0111171C074C089
:103DD0009F3F19F09F5F9093D401181624F40E941E
:103DE000411D8093D6018091D60187FF05C00E94B6
:103DF000411D81958093D6011C1624F40E94411D1B
:103E00008093D7018091D70187FF05C00E94411D93
:103E100081958093D7016091D601662331F1C091DD
:103E2000D701CC2311F1062E000C770B880B990BD0
:103E30000E94322223E333E343E35FE30E949622AE
:103E40000E94FA216093D6016C2FCC0F770B880B60
:103E5000990B0E94322223E333E343E35FE30E94A2
:103E600096220E94FA216093D7011D1624F40E9425
:103E70008A1D8093D8018091D80187FF05C00E94D8
:103E80008A1D81958093D801111624F40E948A1D01
:103E90008093D9018091D90187FF05C00E948A1DB6
:103EA00081958093D901DF91CF911F910C94B01E21
:103EB0009F3F09F08FCFA0CFDF91CF911F91089541
:103EC000E5EDF1E085E0DF011D928A95E9F71092BA
:103ED000D4011092D3010895833081F128F4813008
:103EE00059F08230D1F00895853009F449C0B8F115
:103EF000863009F456C0089580911501262F30E0D0
:103F0000280F311D2F3F310524F4680F60931501F0
:103F100008958FEF80931501089580911401262F45
:103F200030E0280F311D2F3F310524F4680F6093D6
:103F3000140108958FEF8093140108958091130167
:103F4000262F30E0280F311D2F3F310524F4680F54
:103F50006093130108958FEF80931301089580916A
:103F60001201262F30E0280F311D2F3F310524F498
:103F7000680F6093120108958FEF809312010895E6
:103F800080911101262F30E0280F311D2F3F310580
:103F900024F4680F6093110108958FEF809311014D
:103FA000089580911001262F30E0280F311D2F3FFA
:103FB000310524F4680F6093100108958FEF80930A
:103FC00010010895833011F128F4813049F08230D6
:103FD00091F00895853081F120F18630C1F1089586
:103FE00080911501681720F4861B809315010895B0
:103FF00010921501089580911401681720F4861B12
:104000008093140108951092140108958091130172
:10401000681720F4861B80931301089510921301F2
:10402000089580911201681720F4861B8093120175
:10403000089510921201089580911101681720F4DB
:10404000861B8093110108951092110108958091AB
:104050001001681720F4861B8093100108951092B8
:10406000100108950F931F938D3109F46BC008F070
:104070003FC08E3009F47DC0C0F4873009F46EC0B3
:1040800068F4863009F0AFC08091CC01817F8E7FCB
:104090008093CC0181E08093DB01A6C0883009F4D5
:1040A00058C08B3009F49BC09EC0863109F497C07C
:1040B00078F4803109F470C0813109F094C00E9415
:1040C0006B1490910D0181E0892780930D0187C0C9
:1040D000893109F484C08B3109F085C08091CC010D
:1040E00081FB222720F991E0922790FB81F94AC0B9
:1040F000853309F45BC048F4873209F457C008F4EB
:104100005AC0893209F452C06EC0833438F48A33FD
:1041100008F067C0883309F462C065C0833409F4CD
:1041200045C0883409F05FC00E946B140FEF13ED97
:1041300020E3015010402040E1F700C000000E9441
:10414000721B4DC00E94B4210E94020F0E94F8070A
:1041500046C00E94261D0E94381D41C09091CC018E
:10416000892F817090FF12C0917F9E7F9093CC0128
:104170003BC08091CC0182FB222720F991E092275D
:1041800090FB82F98093CC01992349F18091CC0175
:1041900081608093CC0123C08091CC0183FB2227D6
:1041A00020F991E0922790FB83F9ECCF61E070E079
:1041B00080E090E010C08D5141E050E060E070E0A0
:1041C0008A019B0104C0000F111F221F331F8A9513
:1041D000D2F7C901B8010E9422180E946B1481E035
:1041E00003C08953E9CF80E01F910F91089580E0CB
:1041F00008950C94F720CF93C82F8091DB01813074
:1042000079F018F08230E9F187C0E0910E01F09169
:104210000F018081813169F0823209F07FC009C0CD
:10422000E0910E01F0910F018081813111F0823215
:1042300061F48C2F0E94F920811104C08C2F0E9400
:1042400032201DC081E090E01AC08C2F0E94F72020
:10425000811114C0C43179F048F4CB3079F0C03109
:1042600009F060C082E08093DB0108C0C93219F018
:10427000C83321F057C01092DB0154C081E0817037
:1042800053C0C93289F118F5C43171F1A8F4C730AF
:1042900009F046C08AE08093150194E190931401DF
:1042A00093E0909313018093120188E080931101B1
:1042B00088E28093100134C0CE51C63088F5EC2FCF
:1042C000F0E0E65DFE4F80818093DA0129C0CE34B4
:1042D000E9F020F4CB3421F56AE013C0C13579F060
:1042E000C235F1F461E00DC08091DA01882319F044
:1042F0001092DA0115C081E08093DB0115C061E006
:1043000006C08091DA010E946C1F0AC06AE08091A9
:10431000DA010E94E21F04C01092DB0180E004C0B9
:1043200081E002C080E0ABCFCF910895E1E8F0E0FA
:104330008081886080838081816080838FB7F894DA
:1043400093E09093890090ED909388008FBF08953B
:10435000EFE6F0E08081826080830895EFE6F0E090
:1043600080818D7F80830895EFE6F0E0908182E088
:104370008927808308951F920F920FB60F92112400
:104380002F933F934F935F936F937F938F939F935D
:10439000AF93BF93EF93FF938091DC019091DD0188
:1043A00001969093DD018093DC01811103C082E0CE
:1043B0000E94F807E091DD01E695E695F0E0E05215
:1043C000FA4FE4918091DC018E1303C080E00E94DB
:1043D000F807FF91EF91BF91AF919F918F917F91DE
:1043E0006F915F914F913F912F910F900FBE0F9062
:1043F0001F9018950E9401226894B1110C9490228C
:1044000008950E94752288F09F5798F0B92F992738
:10441000B751B0F0E1F0660F771F881F991F1AF0AF
:10442000BA95C9F714C0B13091F00E948F22B1E063
:1044300008950C948F22672F782F8827B85F39F062
:10444000B93FCCF3869577956795B395D9F73EF448
:1044500090958095709561957F4F8F4F9F4F0895F0
:10446000E89409C097FB3EF490958095709561950E
:104470007F4F8F4F9F4F9923A9F0F92F96E9BB27C4
:104480009395F695879577956795B795F111F8CF40
:10449000FAF4BB0F11F460FF1BC06F5F7F4F8F4FAB
:1044A0009F4F16C0882311F096E911C0772321F0A1
:1044B0009EE8872F762F05C0662371F096E8862F39
:1044C00070E060E02AF09A95660F771F881FDAF790
:1044D000880F9695879597F9089557FD9058440F42
:1044E000551F59F05F3F71F04795880F97FB991F53
:1044F00061F09F3F79F08795089512161306140610
:10450000551FF2CF4695F1DF08C01616170618069C
:10451000991FF1CF86957105610508940895E89477
:10452000BB2766277727CB0197F908950E94A92218
:104530000C941A230E940C2338F00E94132320F0BD
:10454000952311F00C9403230C94092311240C944B
:1045500090220E946D2270F3959FC1F3950F50E059
:10456000551F629FF001729FBB27F00DB11D639F25
:10457000AA27F00DB11DAA1F649F6627B00DA11DCB
:10458000661F829F2227B00DA11D621F739FB00D71
:10459000A11D621F839FA00D611D221F749F3327E1
:1045A000A00D611D231F849F600D211D822F762F7A
:1045B0006A2F11249F5750409AF0F1F088234AF057
:1045C000EE0FFF1FBB1F661F771F881F91505040C3
:1045D000A9F79E3F510580F00C9403230C94902280
:1045E0005F3FE4F3983ED4F3869577956795B7954A
:1045F000F795E7959F5FC1F7FE2B880F911D969564
:10460000879597F9089597F99F6780E870E060E0D3
:1046100008959FEF80EC089500240A94161617065B
:1046200018060906089500240A94121613061406A3
:1046300005060895092E0394000C11F4882352F006
:10464000BB0F40F4BF2B11F460FF04C06F5F7F4FBE
:104650008F4F9F4F089597FB072E16F4009407D0B5
:1046600077FD09D00E94452307FC05D03EF49095C4
:1046700081959F4F0895709561957F4F0895EE0F36
:10468000FF1F0590F491E02D0994AA1BBB1B51E17B
:1046900007C0AA1FBB1FA617B70710F0A61BB70BB2
:1046A000881F991F5A95A9F780959095BC01CD0157
:1046B0000895F999FECF92BD81BDF89A992780B5EA
:1046C0000895A8E1B0E042E050E00C947C23262F4E
:1046D000F999FECF1FBA92BD81BD20BD0FB6F894E7
:1046E000FA9AF99A0FBE019608950E946723272F20
:1046F0000C946823DC01CB01FC01F999FECF06C0C4
:10470000F2BDE1BDF89A319600B40D92415050408F
:08471000B8F70895F894FFCFFB
:104718002002F907890864083008FC070101BA017A
:1047280028080A03140A3F4D3639A10554051E0509
:10473800E50478049104AA04C304010203040506ED
:044748000708090055
:00000001FF
